:10000000830100308A003B28E50003088301E400F7
:100010002B088100AA0AAC0A00308A002C081F397C
:10002000142087000B1135288207083409340A345C
:100030000C340D340E340E340F340F340F340E34B0
:100040000E340D340C340A340934083406340534C3
:1000500003340234013401340034003400340134F8
:1000600001340234033405340634831264088300F7
:10007000E50E650E090022308400593051202030F1
:1000800084002230512083010730E300F730E20082
:10009000593084006230552083013B2D04068001D5
:1000A000840A0406031D4E280034F00060208000FE
:1000B000840A040870060319003456288312E200EB
:1000C000E31B692863088A006208E20A0319E30A4D
:1000D00082008313631883176208E20A8400000811
:1000E00008008207F6348234A834603484346634DD
:0400F000FA340034AA
:10040200831212232C3A831203190800022A8B1238
:1004120083169B001C141A088B1683120800F00026
:100422000030711870070310F00D0310F10CF10881
:1004320003190800122A2B2A4830D500232A8312D6
:1004420056086E228312D50A55030822D600D60812
:10045200031D202A83120800F401F5010310F30C96
:10046200F20C031C3B2A7008F40771080318710A86
:10047200F5070310F00DF10D72087304031900342F
:100482002F2A3030DA00DB00D50083125A08D90057
:100492005B08DA005508DB001223D5002E3A031957
:1004A200562A55082C3A031D462A8312080030307A
:1004B200DD00DE00D50083125D08DC005E08DD0091
:1004C2005508DE001223D5002E3A03196C2A55086E
:1004D2002C3A031D5C2A831208000712211A071600
:1004E2008312D8000A30D7005130B000A11D7D2AF6
:1004F2005A30B007B00B7B2A64008312581C862A3C
:100502000716211E8A2A07128A2A0712211E8A2A00
:10051200071603148312D80CD70B752A0800D501CD
:10052200D601D701D800A92A0A30F200F3015608F1
:10053200F1005508F0002D225708580784000008E2
:100542000F397407D50075080318750AD600D70A43
:10055200033083125702031C952A5608F1005508EE
:10056200F00008001223BB001223BC001223BD00BE
:100572001223BE001223BF001223C0001223C100A7
:1005820001221223C20012231223C3001223C40029
:100592001223C5001223C6001223C7001223C8006B
:1005A2001223C9001223CA0001221223CB00831294
:1005B200080041306E2254306E220B306E2204301D
:1005C2006E22FF30042B1223D50083169C18E72AD3
:1005D2008312550883169B008312122383169A00F6
:1005E20003108B1B03148B1383161C1555309D00AF
:1005F200AA309D009C141C1103188B179C18FF2A0B
:100602008312550808226E2283121223D500573A0C
:100612000319E42A83125508523A031D08001223D3
:10062200032B192B6400851C182B20111A2B201563
:100632008312871A1E2B211A132B871E222B211E8F
:10064200132BD6011E30B000B00B252B0830D7007B
:10065200640051308312B000A11D332B5A30B00711
:10066200B00B312B03108312D60C211E3B2B871AA1
:100672003E2B3D2B871E3E2BD617D70B292B5130F5
:10068200B000A11D492B5A30B007B00B462B831284
:10069200560808006400D701D800083057028312B8
:1006A200031808002111581821150310A11C6E2BE4
:1006B200A80CA90C211D5F2B0130602B0030F0002B
:1006C200031C652B0130662B0030F00603196D2BDD
:1006D2008430A8060830A90603108312D80CA11F83
:1006E200772B20302A0203187B2B722B3A302A02F6
:1006F200031C772BAA01211D912BAE0A211F9A2BD5
:100702002E08053A031D9A2BA11F8C2B20302A029A
:100712000318902B872B3A302A02031C8C2BAA0138
:10072200A11B952BC930962BE630AB008030A10679
:10073200AE01D70A0830570203180800532B1330B2
:100742006E22D501550FA62BB12B8312D601AB2BEE
:100752006400D60A560FA92BD50A550FA72BB22B28
:100762008312D501D50A0319C82B6400851C201EEB
:10077200BE2BD501D50A2015C12B201EC12B20115D
:10078200D601203056020318B32BD60AC22B1B30D7
:100792000822F000701CCF2B2014D12B83122010C2
:1007A2001B3083120822F0007019A01CDA2BA0174C
:1007B200DC2B8312A0138312DF035F0FE42B1630AE
:1007C2000822DF008312DF08031DF22B20300822EB
:1007D200F000F01B2010213083120822F000F01BE1
:1007E200A013153083120822F000700FFB2B033088
:0E07F200AD00052C1530831208222D06031DC4
:10080000032CAD01052C8312AD0A83120515A11727
:10081000831681158112C930831281008B17FF3036
:10082000A900A800A1101D300822D5008312D50808
:100830007E3003191E2C4B23D503162C4B23A114F9
:100840002117AE01D501831255080822D600D50A1A
:1008500055080E3A031D302CAD08031D302CD60A66
:10086000831256084B2355080E3A0319462C232CA5
:10087000D50A55030822D6005508153A031D432C06
:100880002D0B432CD60A831256084B23831255088E
:10089000153A03194F2C01302D020318382C023061
:1008A0002D02031C5C2CAE304B2392304B2388303E
:1008B0004B238A304B2383122D08023A031D672CE9
:1008C00064304B2340304B2363304B2383122D087D
:1008D000033A031D722C64304B2340304B236530A8
:1008E0004B2383122D08043A031D7D2C66304B23C5
:1008F00040304B2367304B2383122D08053A031DEC
:10090000872C68304B2340304B2369304B23033016
:1009100083124B23F0304B23A11EB42C3E304B23CB
:10092000D50100308A008312550871200038031960
:10093000A52C00308A008312D50A55037120F000DF
:100940000310700C83124B23912C80308312D5003E
:10095000D50A55030822D600D608831203192A2D7A
:1009600056084B238312A82C213083124B23D50128
:10097000083055020318C42C831255083B3E8400EE
:1009800000084B23D50AB82C1E30831208224B23B3
:10099000D501093055020318D52C83125508433E62
:1009A000840000084B23D50AC92C1F30831208226B
:1009B0004B23201CFB2CD501033055020318E82CD7
:1009C00083125508593E840000084B23D50ADC2CBD
:1009D0002F3083124B23D501033055020318FB2C13
:1009E000831255085C3E840000084B23D50A03306F
:1009F0005502031CF02C8312A01F162D2F304B2301
:100A000041304B233D304B232708303E4B232608F3
:100A1000303E4B232508303E4B232408303E4B23E9
:100A20002308303E4B232208303E4B2320308312D4
:100A3000D5001F2D831256087F394B238312D50A08
:100A400055030822D600D6080319292DDF080319FB
:100A50001A2D8312A110FF30A906A80629084B23DE
:100A600028084B2321137E304B237E304B23051166
:100A70008B1311306E2A0830D300D40164008B012F
:100A80008B160A3098000730990083168113FF30C7
:100A900097000230950020308700831220160A301C
:100AA0008316850083122011051405110530D1002D
:100AB000D201A1152116D001D00A64008312520878
:100AC0005104031D792DA116A023A1125308D100B2
:100AD0005408D2000310D30DD40D0730540209304E
:100AE00003195302031C782D0830D3000730D400BB
:100AF0008312CF0F812D1030A106211E812D0830C9
:100B0000A1061223CC00243A03198C2D4C08213A5B
:100B1000031D5D2DDA225D2D83121223473A031D3A
:100B20005D2D83121223503A031D5D2D831285190A
:100B30009A2D2114CF01D0080319A02D1C22831255
:100B4000D0011223CC00563A0319A019B02D12235C
:100B5000543A031D5D2D1223473A0319652F5D2D6D
:100B600083124C08473A031DBE2D1223473A031D3A
:100B70005D2D1223413A0319C72E5D2D4C08523AC0
:100B8000031D5D2D12234D3A031D5D2D1223433AA3
:100B9000031D5D2D8312A015013085061223D10897
:100BA0000319D203D103B90A0319BA0A0122122385
:100BB000563A0319E12E831205141223B32212238D
:100BC0005822012242221C308312082200380319C5
:100BD000FB2D3C30F200F3011C300822F000F10143
:100BE0002D2275083A02031DF72D74083902031CE3
:100BF000BF2E2114BF2E5C30831290227008B700E4
:100C00007108B800593090227008B5007108B6001C
:100C100019300822F000F1017108803AF20038081A
:100C2000803A7202031D162E37087002031C282E0C
:100C30003C308312F200F30118300822F000F10179
:100C40002D227408B3007508B400B101B2019B2EC7
:100C500014308312AF001A300822F000F10171083D
:100C6000803AF2003808803A7202031D392E3708A4
:100C700070020318412E173083120822B300B4010A
:100C8000632E1A3083120822F200F3011730082273
:100C9000F000F1012D227408F0007508F100380809
:100CA000F3003708F20072277408B3007508B40027
:100CB0003808F3003708F200FA30F0000030F10194
:100CC00072277408AF07513083122F02031C6A2E5B
:100CD0005030AF00600A0319610A031D732E3508F6
:100CE000E0003608E10060083502B1006108031C2D
:100CF000610A3602B200B21F852E35086002B100CB
:100D00003608031C360A6102B2003208803AF0004D
:100D100080307002B53003193102031C9C2E6830FC
:100D2000F0000130F10031087002B1003208031CFC
:100D3000320A7102B20083122F08F000F10171082B
:100D4000803AF2003208803A7202031DA92E31085F
:100D500070020318B22E00303A020630031939022D
:100D60000318BA2E3A083402031DB82E390833028C
:100D70000318C02E21143508E0003608E100831264
:100D8000211C5D2DA0232110B901BA015D2D831214
:100D9000A014013085061223A019D52ED1080319FD
:100DA000D203D103B90A0319BA0A83120122B3226A
:100DB00012231223303A0319E12E3B082C3A031D6B
:100DC000E32E05105D2D831205141223012201224A
:100DD000A201A301A401A501A601A7011223CD0030
:100DE000CC012D3A0319E32D83122608A70025080C
:100DF000A6002408A5002308A4002208A30021308F
:100E0000F1004D08D03E1022CE00643083124E0215
:100E1000031C2A2F9C30CE07A30A0A302302031C8E
:100E2000052FF630A307A40A0A302402031C052F5D
:100E3000F630A407A50A0A302502031C052FF63058
:100E4000A507A60A0A302602031C282FF630A6079B
:100E5000A70A052F0A30F1004E0887274C07A20089
:100E60000A302202031C532FF630A207A30A0A30CD
:100E70002302031C532FF630A307A40A0A302402CE
:100E8000031C532FF630A407A50A0A302502031CC1
:100E9000532FF630A507A60A0A302602031C532F4B
:100EA000F630A607A70A83124E08CC000A304C027F
:100EB000031C5D2FF630CC07562F1223CD002C3AA1
:100EC0000319E32D4D082E3AF22E83122017122318
:100ED0004222831212234D3A8312031D6A2F1223DA
:100EE0005822E32DF601F11F7C2FF009F00A0319B7
:100EF000F103F1097617F61773088039F606F31F28
:100F0000BE2FF209F20A0319F303F309BE2FF00012
:100F1000F4010310FD307107031CAE2FF301F03014
:100F20007105031D962F0430F300F10EF20103103A
:100F3000F30AF10D031C982FF10C710870020318CD
:100F4000F000F20DF30B9C2FF41FA82FF209F20A08
:100F50007208F41F0800F009F00A0800F10C0318E9
:100F6000B72FF10C031CF0010310F00C031C03104D
:100F70007008F200F001F00DA42FF601F401F50164
:100F800072087304031DC72FF001F10100341F30F4
:100F9000F6040310F60AF20DF30D031CCA2FF30C2E
:100FA000F20C73087102031DD72F72087002031C24
:100FB000DF2F7208F0027308031C730AF102F40DAC
:100FC000F50DF60BF61ACF2FF61FEB2FF409F40AE6
:100FD0000319F503F5097408F2007508F300761F8C
:100FE0000034F009F00A0319F103F1090034303438
:100FF000303430343034303430340134FF34FF3462
:02400E00CA3BAB
:104200008200A0008A00A400B000A20060009C0010
:104210009E0086008200980098006000A4008A003A
:1042200098008200B20040006000030002005A00C3
:10423000140003003200010000003C002F003E008B
:10424000000000000000000000000000000000006E
:10425000000000000000000000000000000000005E
:10426000000000000000000000000000000000004E
:10427000000000000000000000000000000000003E
:10428000000000000000000000000000000000002E
:10429000000000000000000000000000000000001E
:1042A000000000000000000000000000000000000E
:1042B00000000000000000000000000000000000FE
:1042C00000000000000000000000000000000000EE
:1042D00000000000000000000000000000000000DE
:1042E00000000000000000000000000000000000CE
:1042F00000000000000000000000000000000000BE
:10430000610070007200730074007200610063004D
:104310006B00650072002D0030002E00310031006E
:104320002D003100360066003600330036000000F4
:00000001FF
